S31508000000C815002099010008A5010008A7010008E5
S31508000010A9010008AB010008AD01000800000000B6
S31508000020000000000000000000000000AF0100080A
S31508000030B101000800000000B3010008B50100087E
S31508000040B7010008B7010008B7010008B7010008A2
S31508000050B7010008B7010008B7010008B701000892
S31508000060B7010008B7010008B7010008B701000882
S31508000070B7010008B7010008B7010008B701000872
S31508000080B7010008B7010008B7010008B701000862
S31508000090B7010008B7010008B7010008B701000852
S315080000A0B7010008B7010008B7010008B701000842
S315080000B0B7010008B7010008B7010008B701000832
S315080000C0B7010008B7010008B7010008B701000822
S315080000D0B7010008B7010008B7010008B701000812
S315080000E0B7010008B7010008B701000800F002F8D8
S315080000F000F043F80AA090E8000C82448344AAF171
S315080001000107DA4501D100F038F8AFF2090EBAE86E
S315080001100F0013F0010F18BFFB1A43F0010318472D
S31508000120E051000000520000103A24BF78C878C198
S31508000130FAD8520724BF30C830C144BF04680C60DF
S31508000140704700000023002400250026103A28BF27
S3150800015078C1FBD8520728BF30C148BF0B6070472B
S315080001601FB500F07FF804000020002104F096FD7A
S31508000170401C60601FBD10B510BD00F0BBF81146ED
S31508000180FFF7EEFF04F0A4F900F0D9F803B4FFF77F
S31508000190F2FF03BC00F0DCF80A498D460A4880479E
S315080001A00A480047FEE7FEE7FEE7FEE7FEE7FEE74A
S315080001B0FEE7FEE7FEE7FEE705480649064A074B5F
S315080001C070470000C8150020A11C0008ED000008B3
S315080001D0C80F0020C8150020C8110020C81100202B
S315080001E010B500F03FF8001D10BD00BFB14A000071
S315080001F010B50446FFF7F4FF0068005D000704D554
S31508000200DF2C02D0A4F1200010BD204610BD4FF00F
S31508000210000200B5134694469646203922BFA0E848
S315080002200C50A0E80C50B1F12001BFF4F7AF090754
S3150800023028BFA0E80C5048BF0CC05DF804EB890045
S3150800024028BF40F8042B08BF704748BF20F8022B88
S3150800025011F0804F18BF00F8012B704770477047A0
S315080002607047000000487047840F00200048704718
S31508000270640F00204FF0013C50F8042B51F8043B62
S315080002809A4221D1A2EB0C03934313EACC1317D15C
S3150800029050F8042B51F8043B9A4215D1A2EB0C03F3
S315080002A0934313EACC130BD150F8042B51F8043BB3
S315080002B09A4209D1A2EB0C03934313EACC13DBD081
S315080002C04FF00000704700BFD01A01BAB1FA81F1A9
S315080002D001F0180122FA01F0CB40C1F12001DBB28E
S315080002E0C0B2C01A2CFA01F3D11A914311EAC3110C
S315080002F0E6D170477546FFF7B9FFAE460500694671
S31508000300534620F00700854618B020B5FFF754FF7E
S31508000310BDE820404FF000064FF000074FF00008F8
S315080003204FF0000B21F00701AC46ACE8C009ACE879
S31508000330C009ACE8C009ACE8C0098D46704710B5DD
S315080003400446AFF300802046BDE81040FFF71EBF05
S3150800035001491820ABBEFEE726000200704700BF21
S3150800036000F067FAFCE7000010B500F029FA01284A
S3150800037000D110BD00F064FB00B9FAE70A4800781E
S3150800038001280FD101F0BCFC0849096801F5FA718A
S31508000390884207D300200449087000F0FFFA08B91C
S315080003A000F066FA00BFE4E71C00002020000020E9
S315080003B010B501200449087001F0A2FC0349086041
S315080003C0FFF7D2FF10BD00001C000020200000200F
S315080003D010B500F02FFA00F02BFA01F099FC01F0A5
S315080003E00AFB00F0F3FA00F0DBF9FFF7E1FF10BDB6
S315080003F010B500F01EFA01F0A5FC00F08FFC00F025
S31508000400E3F9FFF7B1FF10BDF0B505460C4600212C
S3150800041033E01C4810F811001A4E06EB41067678B0
S315080004203044401C684348F6A04696FBF0F700FBAC
S31508000430176000BB134810F81100124E06EB410670
S3150800044076783044401C684348F6A04696FBF0F0A0
S315080004502080208800280EDD2088B0F5806F0ADC11
S31508000460084810F811001070064800EB4100407863
S3150800047018700120F0BD481CC1B21229C9D300204A
S31508000480F8E700003E5200083EB56B4601AA02A9ED
S315080004904FF4FA70FFF7B8FF0446012C03D0E221A7
S315080004A046A0FFF75CFF00204E4908604D48143807
S315080004B0006840F400404B491439086001E000F038
S315080004C0B8F948481438006800F400400028F6D106
S315080004D044481438006820F002004249143908607C
S315080004E00846006840F00100086001E000F0A1F944
S315080004F03C481038006800F001000028F6D09DF846
S315080005000400401E01049DF80000401E41EA005008
S31508000510BDF80810491E08433249083108603148B9
S315080005201438006820F001002E491439086001E0EB
S3150800053000F07FF92B481038006800F00100002809
S31508000540F6D12948006840F0010027490860264886
S315080005501C30006820F0010023491C31086022483D
S315080005600C30006840F001001F490C31086000207B
S315080005701D494031086000211B48443001601A4873
S31508000580001D006820F001001749091D086016487B
S315080005901430006820F0010013491431086012482D
S315080005A01C30006840F001000F491C3108600E48F5
S315080005B0006820F001000C4908603EBD2E2E5C2E16
S315080005C02E5C2E2E5C2E2E5C536F757263655C4115
S315080005D0524D434D335F53544D333246315C63615C
S315080005E06E2E6300146400400066004010B5014694
S315080005F000201F4B1B6803F00303002B36D01D4B4E
S315080006001B6840F2FF7404EA535240F267639A4249
S3150800061026D10120174B08331B680B70154B08337E
S315080006201B681B0A4B70134B08331B681B0C8B701B
S31508000630104B08331B681B0ECB700E4B0C331B6814
S315080006400B710C4B0C331B681B0A4B71094B0C3393
S315080006501B681B0C8B71074B0C331B681B0ECB716D
S31508000660034B1B6843F02003014C236010BD0000B8
S315080006700C640040B065004070B504460D4622483B
S31508000680006800F08060B0F1806F04D040F221115C
S315080006901EA0FFF764FE2748006800F00100254900
S315080006A00860084600682449084322490860081D6E
S315080006B00560E0780006A17840EA0140617840EAE2
S315080006C00120217808431B4908310860E0790006B3
S315080006D0A17940EA0140617940EA0120217908437D
S315080006E014490C3108601348006840F001001149AC
S315080006F0086001E000F09DF80348006800F080609B
S315080007000028F7D070BD0000086400402E2E5C2E2D
S315080007102E5C2E2E5C2E2E5C536F757263655C41C3
S31508000720524D434D335F53544D333246315C63610A
S315080007306E2E630080650040000020FC70470000B4
S315080007400A49097831B1012906D0022906D00329B8
S3150800075008D105E0402007E0082005E0002003E076
S31508000760002001E0402000BF00BF704724000020A1
S315080007700A49097831B1012906D0022906D0032988
S3150800078008D105E0402007E0082005E0002003E046
S31508000790002001E0402000BF00BF70472400002071
S315080007A010B501F0C7FDFFF76FFE01200349087079
S315080007B001F060FB00200149087010BD24000020EC
S315080007C010B501F0C5FD10BD10B50B48FFF70EFFBB
S315080007D0012804D109490870074801F0C3FD0648F5
S315080007E001F072FB012805D100200449087002486F
S315080007F001F0B8FD10BD00007002002024000020A2
S3150800080070B505460C4609480078012803D1E1B2BF
S315080008102846FFF731FF0548007818B9E1B228469F
S3150800082001F0B8FB01F024FE70BD00002400002092
S315080008307047704710B500F001F810BD72B67047E2
S3150800084062B670472DE9F04104460D4616462F4616
S31508000850A04605E017F8010B08F8010BFFF7E9FFBA
S31508000860301EA6F101018EB2F4DCBDE8F08100006D
S3150800087010B501F0C4F800B910BDFFF75FFF01F02D
S315080008805BFA01F0B4F8064908400649086001F029
S31508000890AEF84468FFF7D4FFA04700BFECE70000B6
S315080008A080FFFF1F08ED00E010B50E4890F82402FF
S315080008B0012802D10B4802F00BFF01F021FA00F1E2
S315080008C0640404E001F01CFAA04200D905E04021C6
S315080008D0054801F051FA0028F4D000BF034803F098
S315080008E05DFA10BD4800002000440040C84C0008CE
S315080008F010B50446044890F82402012802D102489B
S3150800090002F0E6FE10BD00004800002010B50446BF
S31508000910114890F8240201280CD10F49204603F00B
S31508000920C8F8002806DA00200B4981F82402084690
S3150800093002F0CEFE0BE02178084801F097FA00BFD6
S315080009408021064801F018FA0028F9D0641C20789E
S315080009500028F0D110BD00004800002000440040E7
S3150800096010B50020064981F824020A2205A1044888
S3150800097002F0D2FF18B90120014981F8240210BDFE
S31508000980480000202F626F6F746C6F672E7478743E
S315080009900000000000487047C84C000810B5FFF773
S315080009A00FFF012801D1002010BD0748007808B1C3
S315080009B00020F9E700F02AF8012802D10249087058
S315080009C0F2E70020F0E700002800002010B500201C
S315080009D005490870054902F089FF04461CB17721CC
S315080009E003A0FFF7BCFC10BD28000020B0020020C1
S315080009F02E2E5C2E2E5C2E2E5C2E2E5C536F757260
S31508000A0063655C66696C652E6300000000B589B095
S31508000A10202101A8FFF7FBFB01A9084803F044F9C8
S31508000A2048B9019838B19DF80C0000F0100010B9CB
S31508000A30012009B000BD0020FBE70000C84C0008F3
S31508000A400348007808B9012070470020FCE7000039
S31508000A502800002070B5044604F00F0000F13005A8
S31508000A60092C02DDE81DC5B203E02846FFF7C0FBE6
S31508000A70C5B2284670BD70B505460C462811FFF765
S31508000A80E9FF207005F00F00FFF7E4FF6070002013
S31508000A90A070204670BD2DE9F041064600270025C6
S31508000AA01AE0705DFFF7A4FBC4B2302C05DB462CB8
S31508000AB003DC392C04DD412C02DA0020BDE8F08184
S31508000AC0A4F13000C4B2092C01DDE01FC4B204EB66
S31508000AD00710C7B2681CC5B2022DE2DB3846EDE73F
S31508000AE010B503461A4600BF491C0A20B2FBF0F2AD
S31508000AF0002AF9D1002008701A4600BF491E0A20AC
S31508000B00B2FBF0F400FB1420303008700A20B2FB68
S31508000B10F0F2002AF2D1084610BD10B50446207836
S31508000B20FFF766FB53280AD1FFF75AFB006861787E
S31508000B30405C202801D1012000E0002008B90320EC
S31508000B4010BD6078312801D10020F9E76078322895
S31508000B5001D10120F4E76078332801D10220EFE7BC
S31508000B600320EDE72DE9F04704460D4617464FF0FA
S31508000B70000905B124B940F2312150A0FFF7EFFB77
S31508000B802046FFF7CAFF8246BAF1030F02D10020BA
S31508000B90BDE8F087204600F09FF810B94FF0FF3007
S31508000BA0F6E7BAF1000F06D0BAF1010F25D0BAF16F
S31508000BB0020F7FD14BE0A41C2046FFF76CFF80464E
S31508000BC0A41C2046FFF767FF00022860A41C2046E5
S31508000BD0FFF761FF296808442860A41CA8F10309E7
S31508000BE057B1002606E02046FFF755FFB855A41C66
S31508000BF0701C86B24E45F6DB5DE0A41C2046FFF766
S31508000C004AFF8046A41C2046FFF745FF00042860DB
S31508000C10A41C2046FFF73FFF296801EB0020286047
S31508000C20A41C2046FFF737FF296808442860A41C3F
S31508000C30A8F1040957B1002606E02046FFF72BFF66
S31508000C40B855A41C701C86B24E45F6DB33E0A41CCE
S31508000C502046FFF720FF8046A41C2046FFF71BFF0F
S31508000C6000062860A41C2046FFF715FF296801EB3B
S31508000C7000402860A41C2046FFF70DFF296801EBF9
S31508000C8000202860A41C2046FFF705FF29680844B1
S31508000C902860A41CA8F105095FB1002607E009E051
S31508000CA02046FFF7F8FEB855A41C701C86B24E45C0
S31508000CB0F6DB00E000BF00BF484669E72E2E5C2E33
S31508000CC02E5C2E2E5C2E2E5C536F757263655C66E9
S31508000CD0696C652E6300000070B504460025A41CE7
S31508000CE02046FFF7D8FE0646A819C5B2A41C00BFC1
S31508000CF02046FFF7D0FE2844C5B2701E86B2A41C53
S31508000D00012EF5DCE843C5B22046FFF7C4FEA8422B
S31508000D1001D0002070BD0120FCE7000070B500245A
S31508000D20D248007800282BD0D0480078012828D14E
S31508000D30FFF716FECEA0FFF7E9FDD6A0FFF7E6FD02
S31508000D40FFF728FE064601223146DC4802F0E4FD9C
S31508000D5030B1DBA0FFF7DAFD0120FFF7C9FD70BD52
S31508000D60D9A0FFF7D3FDDAA0FFF7D0FDE1A0FFF782
S31508000D70CDFD0020EB49086048600220BB49087099
S31508000D8072E1BA48007802287ED1CC4AC101E64809
S31508000D9002F0A9FC0546E54890F83A02C009002881
S31508000DA00CDDC7A0FFF7B2FD0220FFF7A1FDC3487F
S31508000DB002F08EFC0020AD490870D0E7A5B10022EC
S31508000DC0DB49D948FFF7CEFE0446601C60B9BCA0D3
S31508000DD0FFF79CFD0320FFF78BFDB84802F078FC6F
S31508000DE00020A2490870BAE7002C1BDDCD484068F0
S31508000DF038B9CD48D0F88001CA4908600846446029
S31508000E0010E0C948D0F88001C6490968884204D26A
S31508000E10C548D0F88001C3490860C24840682044E4
S31508000E20C0494860C148D0F83C12D0F84002814217
S31508000E3001D1012000E000200028A1DD00219F4803
S31508000E4002F07CFC60B19EA0FFF760FD0420FFF76E
S31508000E504FFD9A4802F03CFC0020844908707EE762
S31508000E6099A0FFF753FDB3A0FFF750FDAD494868B9
S31508000E70B349FFF735FEB248FFF748FDB1A0FFF7C3
S31508000E8045FDA849096800E039E0080EAC49FFF7B6
S31508000E90F2FDA4490968C1F30740A949891CFFF76F
S31508000EA0EAFDA0490988C1F30720A549091DFFF7EE
S31508000EB0E2FD9C490878A249891DFFF7DCFDA04898
S31508000EC0FFF724FDA6A0FFF721FD964A5168106892
S31508000ED000F085FD60B97AA0FFF718FD0520FFF739
S31508000EE007FD764802F0F4FB00206049087036E7F3
S31508000EF075A0FFF70BFD03205C490870B4E05B485A
S31508000F0000780328FAD16D4A4FF48071864802F0BA
S31508000F10EAFB0546854890F83A02C00900280CDD28
S31508000F2090A0FFF7F3FC0220FFF7E2FC634802F00B
S31508000F30CFFB00204D49087011E7ADB17C4A803AD5
S31508000F407B497948FFF70EFE0446601C60B98EA0FF
S31508000F50FFF7DCFC0320FFF7CBFC584802F0B8FB90
S31508000F60002042490870FAE6002C4BDD8FA0FFF7F7
S31508000F70CDFC73492046FFF7B3FD7148FFF7C6FC61
S31508000F808EA0FFF7C3FC6849D1F88011080E6C499A
S31508000F90FFF771FD6449D1F88011C1F3074068492C
S31508000FA0891CFFF768FD6049B1F88011C1F3072075
S31508000FB06349091DFFF75FFD5B4991F880016049A8
S31508000FC0891DFFF758FD5E48FFF7A0FC64A0FFF7F0
S31508000FD09DFC554901F58072D1F88001214600F043
S31508000FE012FD60B936A0FFF791FC0620FFF780FCDA
S31508000FF0324802F06DFB00201C490870AFE632A0AB
S31508001000FFF784FC4948D0F83C12D0F840028142E8
S3150800101001D1012000E00020002825DD6DA0FFF7A2
S3150800102075FC00F0D3FC60B925A0FFF76FFC07201C
S31508001030FFF75EFC214802F04BFB00200B490870C5
S315080010408DE621A0FFF762FC69A0FFF75FFC1B484D
S3150800105002F03EFB6CA0FFF759FC0020034908701C
S31508001060FFF722FCFFF704FC00BF78E62800002003
S315080010704669726D77617265207570646174652062
S3150800108072657175657374206465746563746564E7
S315080010900A0D00004F70656E696E67206669726D8D
S315080010A0776172652066696C6520666F7220726565
S315080010B06164696E672E2E2E00000000E40400208D
S315080010C04552524F520A0D004F4B0A0D00000000C0
S315080010D05374617274696E67207468652070726FE4
S315080010E06772616D6D696E672073657175656E638C
S315080010F0650A0D0050617273696E67206669726DC4
S31508001100776172652066696C6520746F206F6274FA
S3150800111061696E2065726173652073697A652E2E22
S315080011202E0000002C00002008070020B002002036
S315080011308808002045726173696E67200000000008
S315080011408C0800202062797465732066726F6D20A2
S315080011506D656D6F7279206174203078000000002B
S315080011602E2E2E0052656164696E67206C696E6565
S315080011702066726F6D2066696C652E2E2E4552525A
S315080011804F520A0D00000000496E76616C696420B2
S31508001190636865636B73756D20666F756E642E2E56
S315080011A02E4552524F520A0D0000000050726F67CA
S315080011B072616D6D696E67200000000020627974A7
S315080011C0657320746F206D656D6F72792061742068
S315080011D03078000057726974696E672070726F679D
S315080011E072616D20636865636B73756D2E2E2E00B4
S315080011F0436C6F73696E67206669726D7761726595
S315080012002066696C650A0D004669726D77617265BC
S31508001210207570646174652073756363657373669E
S31508001220756C6C7920636F6D706C657465640A0DF6
S31508001230000000002DE9F04704460E4692461F4678
S31508001240700A4FEA40282068401C38B941462046B3
S3150800125000F03AF910B90020BDE8F087206840454B
S3150800126007D04146204600F04FF904460CB9002045
S31508001270F2E72068311A201D0D18D14600BFFFF786
S31508001280D8FA201D281AB0F5007F09D308F5007191
S31508001290204600F039F904460CB90020DCE7251D84
S315080012A099F8000028706D1C09F101097F1E002FAE
S315080012B0E5D10120D0E7000010B50B480068401CB6
S315080012C028B1094800F0ACF908B9002010BD074854
S315080012D00068401C28B1054800F0A2F908B90020AA
S315080012E0F4E70120F2E700001C0D0020180B00208F
S315080012F02DE9F04104460D46204600F071F80646F1
S315080013006119481E00F06CF80746FF2E01D0FF2F22
S3150800131002D10020BDE8F0813946304600F002F8D7
S31508001320F8E700002DE9F04706460D46AE4202DD15
S315080013300020BDE8F0872848007AB04204DC264839
S3150800134090F89800A84201DA0020F2E700F002F9C6
S315080013502248C06800F0010018B100F0CBF8002060
S31508001360E7E71E48006940F002001C49086130465C
S3150800137000F060F80746284600F05CF882462846E2
S3150800138000F074F85044A0F10109A9EB0700401CCD
S31508001390C0F38F28002413E007EB84200F49486127
S315080013A00846006940F04000086101E0FFF741FA8D
S315080013B00A48C06800F001000028F7D1601C84B212
S315080013C04445E9DB0548006920F002000349086145
S315080013D000F090F80120ACE76452000800200240B3
S315080013E070B5054600241EE0FFF723FA04EB440017
S315080013F00F4951F82000A84213D804EB440051F8CD
S31508001400200004EB44010A4A02EB810149680844BA
S31508001410A84206D904EB4400114601EB8000007A85
S3150800142070BD601CC4B20D2CDED3FF20F8E70000A7
S315080014306452000870B50546002410E0FFF7F9F974
S3150800144004EB4400084901EB8000007AA84204D165
S3150800145004EB440051F8200070BD601CC4B20D2C8A
S31508001460ECD34FF0FF30F7E76452000870B5054635
S31508001470002411E0FFF7DDF904EB4400084901EB0D
S315080014808000007AA84205D104EB440001EB8000F5
S31508001490406870BD601CC4B20D2CEBD30020F8E781
S315080014A0645200080148006870470000645200084A
S315080014B04FF0FF3002490860024908607047000093
S315080014C0180B00201C0D002070B505460C46C4F309
S315080014D0080008B1002070BD2868A04201D101208B
S315080014E0F9E72C604FF400722146281DFFF7AAF988
S315080014F00120F0E70348006940F0800001490861CF
S31508001500704700000020024070B504460D460E489C
S31508001510844201D10D4C0DE00D480068A84203D164
S31508001520094C0B48056805E0204600F079F808B92B
S31508001530002070BD29462046FFF7C6FF08B90020DF
S31508001540F7E72046F5E700001C0D0020180B0020E1
S315080015506452000803480449486004484860342037
S31508001560C86070472301674500200240AB89EFCD6C
S315080015700021134800680068014411480068406863
S3150800158001440F480068806801440D480068C06837
S3150800159001440B480068006901440948006840692D
S315080015A00144074800688069014405480068D0F886
S315080015B05001014409B9012070470020FCE70000EA
S315080015C0645200082DE9F04104460D4617462046A8
S315080015D0FFF706FFFF2805D06119481EFFF700FF31
S315080015E0FF2802D10020BDE8F081600A46020948BA
S315080015F00068B04206D12B463A4621460648FFF710
S3150800160019FEF0E72B463A4621460448FFF712FE34
S31508001610E9E70000645200081C0D0020180B0020A2
S315080016202DE9F04705464FF001092868FFF7D8FE6F
S315080016308046B8F1FF0F02D10020BDE8F087FFF71A
S3150800164089FF2048C06800F0010018B1FFF752FF73
S315080016500020F2E71B48006940F0010019490861BB
S31508001660002421E0286800EB8406281D50F8247021
S31508001670378001E0FFF7DDF81248C06800F0010086
S315080016800028F7D1380C708001E0FFF7D2F80D4832
S31508001690C06800F001000028F7D13068B84202D0CF
S315080016A04FF0000902E0641C802CDBD300BF05481C
S315080016B0006920F0010003490861FFF71BFF48464F
S315080016C0BBE700000020024008B5002000901C4837
S315080016D00068401C08B9012008BD194840680099EF
S315080016E008440090164880680099084400901448F9
S315080016F0C068009908440090114800690099084498
S3150800170000900F4840690099084400900C48806989
S315080017100099084400900A48C06900990844009056
S315080017200098C04300900098401C0090054909683D
S3150800173001F5A8706A460421FFF744FFCCE70000CC
S315080017401C0D0020645200082DE9F04102460025D0
S315080017500026002000230024002791F803C00CF07F
S315080017600F0591F803C00CF0100CBCF1000F03D064
S3150800177091F802C04CEA050591F800C0BCF1000FCB
S3150800178031D0146800202BE04FF0010C0CFA00F35E
S31508001790B1F800C00CEA03069E4220D183004FF040
S315080017A00F0C0CFA03F7BC4305FA03FC4CEA0404D5
S315080017B091F803C0BCF1280F06D14FF0010C0CFAC2
S315080017C000FCC2F814C00AE091F803C0BCF1480F47
S315080017D005D14FF0010C0CFA00FCC2F810C0401CF1
S315080017E00828D1D31460B1F800C0BCF1FF0F34DD6E
S315080017F0546800202EE000F1080C4FF0010808FAA2
S315080018000CF3B1F800C00CEA03069E4221D183000E
S315080018104FF00F0C0CFA03F7BC4305FA03FC4CEA2D
S31508001820040491F803C0BCF1280F05D100F1080C97
S3150800183008FA0CF8C2F8148091F803C0BCF1480FF6
S3150800184007D100F1080C4FF0010808FA0CF8C2F8A5
S315080018501080401C0828CED35460BDE8F0810000F3
S31508001860F0B50A46002300240021002500F00046B2
S31508001870B6F1004F02D11D4EF16901E01B4E7168A9
S31508001880C0F3034583B200F44016B6F5401F08D1ED
S3150800189021F07061154E766826F07066134F7E60EB
S315080018A012E000F48016B6F5801F06D1032606FA64
S315080018B005F4A14341F0706106E0460D360103FACE
S315080018C006F6B14341F0706122B1460D360103FABE
S315080018D006F6314300F00046B6F1004F02D1034E3A
S315080018E0F16101E0014E7160F0BD000000000140A9
S315080018F0416170470161704700B585B0012108460E
S3150800190000F09CF80121082000F098F84FF4807048
S31508001910ADF8100048208DF8130004A92848FFF7F1
S3150800192013FF4FF40070ADF8100018208DF813005F
S3150800193003208DF8120004A92148FFF705FF0121AD
S315080019404FF4EA10FFF78CFF0121480600F066F80D
S315080019500121480400F062F80121052000F06EF824
S3150800196018208DF813000420ADF8100003208DF818
S31508001970120004A91348FFF7E7FE04208DF81300A8
S315080019800820ADF8100004A90E48FFF7DDFE4FF455
S31508001990614000900020ADF80400ADF80600ADF8EF
S315080019A00800ADF80C000C20ADF80A006946064898
S315080019B000F0F0F90121044800F0D2F905B000BDA5
S315080019C0000C0140000801400044004010B5FFF734
S315080019D07BFE08B9002010BDFFF76EFCFBE770B56B
S315080019E004460D4629462046FFF782FC70BD10B511
S315080019F0FFF758FD10BD10B5FFF75AFD10BD10B51D
S31508001A00FFF7B6FD10BD70B504460D4616463246BC
S31508001A1029462046FFF7D6FD70BD000029B1064AC3
S31508001A20D2690243044BDA6104E0034AD26982436D
S31508001A30014BDA61704700000010024029B1064ADE
S31508001A4092690243044B9A6104E0034A926982430D
S31508001A50014B9A61704700000010024030B5002122
S31508001A600022002400232D4D6D6805F00C0121B1DC
S31508001A70042905D0082923D105E0294D056022E06F
S31508001A80274D05601FE0254D6D6805F47012234D3E
S31508001A906D6805F48034022505EB92421CB9214D88
S31508001AA0554305600BE01D4D6D6805F400351DB105
S31508001AB01C4D5543056002E0194D5543056002E08B
S31508001AC0174D056000BF00BF144D6D6805F0F001A5
S31508001AD00909154D6B5C0568DD4045600F4D6D685D
S31508001AE005F4E061090A104D6B5C4568DD408560C8
S31508001AF00A4D6D6805F46051C90A0B4D6B5C456863
S31508001B00DD40C560054D6D6805F44041890B074DFC
S31508001B106B5CC568B5FBF3F5056130BD0010024086
S31508001B2000127A0000093D00000000201000002085
S31508001B3021B1028842F40052028004E002884DF680
S31508001B40FF731A400280704721B1028842F04002B2
S31508001B50028004E002884FF6BF731A40028070477D
S31508001B600246002013890B400BB1012000E000203B
S31508001B7070470146888970478181704710B50022F1
S31508001B80028802F441520B884C8823438C882343ED
S31508001B90CC8823430C8923434C8923438C892343CC
S31508001BA0CC8923431A430280838B4FF2FF74234068
S31508001BB083830B8A038210BD10B500F001F810BDAF
S31508001BC00CB50020019000903348006840F480303E
S31508001BD03149086000BF3048006800F400300090C2
S31508001BE00198401C0190009818B90198B0F5A06FAB
S31508001BF0F1D12948006800F4003010B101200090A6
S31508001C0001E0002000900098012843D1234800688D
S31508001C1040F01000214908600846006820F00300DB
S31508001C2008600846006840F0020008601A484068E4
S31508001C30194948600846406848600846406840F4C4
S31508001C40806048600846406820F47C104860084672
S31508001C50406840F4E81048600846006840F0807024
S31508001C60086000BF0C48006800F000700028F9D032
S31508001C700948406820F0030007494860084640685C
S31508001C8040F00200486000BF0348406800F00C00BE
S31508001C900828F9D10CBD00000010024000200240BF
S31508001CA010B51348006840F001001149086008465D
S31508001CB04068104908400E494860084600680E49C1
S31508001CC008400B4908600846006820F48020086030
S31508001CD00846406820F4FE0048604FF41F008860FC
S31508001CE0FFF76AFF4FF000600449086010BD000066
S31508001CF0001002400000FFF8FFFFF6FE08ED00E0C6
S31508001D0000B500F01FF80148006800BD3C0000203F
S31508001D1000B500F011F806484FF0E02148610020B0
S31508001D2088610520086100200249086000BD00009E
S31508001D303F1901003C00002000204FF0E021086117
S31508001D40704700004FF0E020006900F4803020B1B1
S31508001D5002480068401C0149086070473C000020A2
S31508001D6021B1828942F40052828104E082894DF6CB
S31508001D70FF731A408281704702460020B1F5007F42
S31508001D8000D100BF13880B400BB1012000E00020F2
S31508001D90704700002DE9F04786B005460E46002438
S31508001DA0A24600BFA1460027B08900B100BF2F4652
S31508001DB02C8A4CF6FF700440F08804432C82AC89C8
S31508001DC04EF6F3100440B0883189084371890843F8
S31508001DD00443AC81AC8A4FF6FF400440B089044303
S31508001DE0AC8201A8FFF73AFE1F48874202D1DDF808
S31508001DF010A001E0DDF80CA0A88900F4004040B16D
S31508001E000AEBCA0000EB0A1031684900B0FBF1F88A
S31508001E1007E00AEBCA0000EB0A1031688900B0FB3C
S31508001E20F1F86420B8FBF0F004012009642101FBF5
S31508001E301089A88900F4004040B1322000EBC9009F
S31508001E40B0FBF1F000F00700044308E0322000EB95
S31508001E5009106421B0FBF1F000F00F0004432C8157
S31508001E6006B0BDE8F087000000380140C1F308025B
S31508001E708280704700200B490880091D0880091DCB
S31508001E800880091D0880091D088040F2712005494F
S31508001E900880081D008842F20C0108430149091D03
S31508001EA0088070470844004001460648008800F04C
S31508001EB0200028B10348001D0088087001207047DB
S31508001EC00020FCE70044004010B50446204800788E
S31508001ED098B92048FFF7E8FF012837D11D48007850
S31508001EE0002833DDFFF70CFF1B49086000201B495B
S31508001EF0087001201649087028E0164A174909781B
S31508001F00491C5018FFF7D0FF012815D1134800784F
S31508001F10401C124908700F4800780978884215D184
S31508001F200E4802780B49491C2046FEF78BFC002018
S31508001F3007490870012010BDFFF7E2FE0649096847
S31508001F406431884202D90020014908700020F2E76E
S31508001F5041000020200F00204400002040000020FF
S31508001F6010B504460A48008800F0800008B9002029
S31508001F7010BD0748001D048001E0FEF75AFC04481E
S31508001F80008800F080000028F7D00120F0E7000064
S31508001F90004400402DE9F04107460C46402C03DD7D
S31508001FA08D2110A0FEF7DBF92046FFF7D9FF06467C
S31508001FB0012E03D091210BA0FEF7D1F900250DE0E3
S31508001FC0FEF737FC785DFFF7CBFF0646012E03D0F8
S31508001FD09A2104A0FEF7C3F9681C85B2A542EFDB77
S31508001FE0BDE8F0812E2E5C2E2E5C2E2E5C2E2E5CED
S31508001FF0536F757263655C41524D434D335F53545D
S315080020004D333246315C756172742E6300000000F0
S3150800201010B50446FF200949C870084A6168906CE3
S31508002020D21D00F077F9054908710021034841716E
S31508002030817108200149A1F8440010BDCC08002090
S3150800204010B5044600BFFEF7FBFC18B9102000F0D7
S315080020501DFA10BD00F014FA012014490870FF207B
S31508002060C870002111480171007940F010010F482D
S3150800207001710021417140790C494871FEF760FBF6
S31508002080C1B20A488171FEF773FBC1B20748C17134
S31508002090FEF76EFB01120548017201214172817239
S315080020A008200249A1F8440000BFD2E7CC08002066
S315080020B010B5044600BF00200549087000F0E0F995
S315080020C0FF200349C8700120A1F8440010BD000094
S315080020D0CC08002000BFFF21084AD1700849916446
S315080020E0002206490A714A718A710722C1F8072037
S315080020F00821024AA2F8441070470000CC080020C4
S31508002100E84C000800BFFF21074AD17000220649A3
S315080021100A714A784A7100228A71CA710A720621BE
S31508002120014AA2F844107047CC08002010B50446AE
S31508002130FEF706FB801E6178884203DA222000F04B
S31508002140A5F910BDFF201049C8700120A1F8440068
S31508002150607830B9FFF73AFC10B9312000F096F9EB
S31508002160EFE76178084A906CA21CFFF74CFC18B997
S31508002170312000F08BF9E4E70348806C6178084465
S315080021800149886400BFDCE7CC08002010B5044686
S31508002190084A6168906CFFF722FC18B9312000F0F4
S315080021A075F910BDFF200349C8700120A1F8440045
S315080021B000BFF6E7CC08002070B50446FEF7C0FA63
S315080021C0451E0D49621C886C2946FFF71CFC18B988
S315080021D0312000F05BF970BDFF200749C870FEF793
S315080021E0AFFA401E0449896C0844034988640120F3
S315080021F0A1F8440000BFEEE7CC08002010B504465D
S31508002200312000F043F910BD10B5044600BFFEF7B3
S315080022102FFBFF200249C8700120A1F8440010BD19
S31508002220CC08002010B5044600BFFF200949C87035
S315080022300021084801714171FEF782FAC1B20548CA
S3150800224081710021C1710172417207200149A1F80B
S31508002250440010BDCC080020FF21044AD170416813
S3150800226091640121A2F8441070470000CC080020B0
S3150800227010B50446FEF764FA401E6178884203DA10
S31508002280222000F003F910BD0B4960688864627863
S315080022900846816C001DFEF7D5FAFF200649C8706E
S315080022A00846806C61780844034988646078401C55
S315080022B0A1F8440000BFE6E7CC08002010B50446A4
S315080022C000BF002000F0E2F810BD000010B504467B
S315080022D0FEF736FA401E6178884203DA222000F0BB
S315080022E0D5F810BD62780A48816C001DFEF7AAFA77
S315080022F0FF200749C8700846806C6178084404497D
S3150800230088646078401CA1F8440000BFE9E7000033
S31508002310CC08002030B50346002403E01878204492
S31508002320C4B25B1C081EA1F10101F7D1146001209B
S3150800233030BD0000002005490870886481F8430014
S31508002340A1F844008870487070470000CC08002047
S315080023500348007808B9002070470120FCE7000010
S31508002360CC08002010B504462078FF2803D1204663
S31508002370FFF766FE60E03D48007801285BD12078CB
S31508002380F4281FD010DCD0283CD006DCC92835D06C
S31508002390CC2847D0CF2849D140E0D1283AD0D228F6
S315080023A034D0F32842D115E0F5380A283ED2DFE8C2
S315080023B000F0050D3D3D3D153D191D212046FFF751
S315080023C085FF37E02046FFF753FF33E02046FFF747
S315080023D043FF2FE02046FFF71BFE2BE02046FFF7C2
S315080023E079FE27E02046FFF769FF23E02046FFF73E
S315080023F089FE1FE02046FFF75BFE1BE02046FFF73D
S31508002400DBFE17E02046FFF791FE13E02046FFF7B4
S3150800241009FF0FE02046FFF7B9FE0BE02046FFF75D
S31508002420F3FE07E02046FFF7E9FE03E0202000F070
S315080024302DF800BF00E010BD0C4890F843000128B5
S3150800244002D1102000F022F80848B0F9440000280C
S3150800245009DD0120054981F843000846B0F9441012
S31508002460C01C00F01FF800BFE5E70000CC080020FC
S315080024700020024981F8430070470000CC0800207C
S315080024800020014948707047CC080020FE21044A04
S31508002490D170114608710221A2F844107047000055
S315080024A0CC08002070B505460C46A1B22846FEF7B2
S315080024B0A7F970BD70B504460D46607801232A4613
S315080024C004F1340101F056F808B1032070BD94F800
S315080024D0321294F8330241EA00204AF6552188421E
S315080024E001D00220F2E794F86D00010694F86C001A
S315080024F041EA004194F86B0041EA002094F86A101A
S31508002500084320F07F400E49884201D10020DDE7CC
S3150800251094F88900010694F8880041EA004194F885
S31508002520870041EA002094F88610084320F07F408F
S315080025300349884201D10020C8E70120C6E7000008
S3150800254046415400024600E0521C107810B110783B
S315080025508842F9D1107870472DE9F74F88B0089866
S315080025600068019001980078303807900798092884
S315080025700AD8019840783A2806D10198801C01901B
S3150800258008990198086001E0002007900021099841
S315080025900160079818B10B200BB0BDE8F08FD14940
S315080025A0079851F820400CB90C20F5E70998046003
S315080025B0207878B1607801F027F8804608F00100A5
S315080025C040B90A9820B108F0040008B10A20E3E7E8
S315080025D00020E1E70020207007986070607800F01E
S315080025E00BFE804608F0010008B10320D4E70A98DC
S315080025F020B108F0040008B10A20CDE74FF0000921
S3150800260049462046FFF756FF054600BF012D21D152
S315080026104FF0000BBBF1000F03D0ABF1010000F047
S31508002620FF0B4FF4DF7000EB0B1104F134000F18A9
S31508002630387978B1F87A0106B87A41EA0041787AA9
S3150800264041EA0020397A40EA010949462046FFF75F
S3150800265031FF0546032D01D101209DE70DB10D205F
S315080026609AE73F20015D94F8400041EA0020B0F562
S31508002670007F01D00D208FE74A20015D94F84B00BA
S3150800268041EA002ABAF1000F0ED194F85B00010660
S3150800269094F85A0041EA004194F8590041EA0020AA
S315080026A094F8581040EA010AC4F81CA04420065DB4
S315080026B0E670012E03D0022E01D00D206CE70AFB2E
S315080026C006FA4120005D0646A07016B1701E30401D
S315080026D008B10D2060E74520015D94F8460041EAFF
S315080026E000202081207A00F00F0008B10D2053E762
S315080026F04720015D94F8480041EA002006900698B4
S3150800270070B994F85700010694F8560041EA00415A
S3150800271094F8550041EA002094F8541008430690AE
S315080027204220015D94F8430041EA00200290029895
S3150800273008B90D2030E702985044218900EB1110A2
S315080027400590DDE90501814201D20D2024E7DDE986
S315080027500510401AA178B0FBF1F00490049808B966
S315080027600D2019E7012540F6F6710498884200D332
S3150800277002254FF6F6710498884200D3032504987B
S31508002780801CA061C4F820900298484460620598AD
S315080027904844E062032D16D1208908B10D20FBE6D6
S315080027A094F86300010694F8620041EA004194F83F
S315080027B0610041EA002094F860100843A062A0690D
S315080027C08000039014E0208908B90D20E4E6606AC9
S315080027D05044A062022D02D1A069400007E0207E85
S315080027E000F00100A16901EB410100EB51000390E3
S315080027F0E169039800F2FF10B1EB502F01D20D20CA
S31508002800CAE64FF0FF3020610020E060032D5CD15E
S31508002810607194F8641094F8650041EA0020484411
S3150800282060616078012304F13401626900F0A2FE58
S31508002830F0BB94F8321294F8330241EA00204AF6C3
S315080028405521884241D13720005D01063620005DBA
S3150800285041EA00413520005D41EA002094F8341031
S3150800286008432149884230D194F81B02010694F89E
S315080028701A0241EA004194F8190241EA002094F844
S3150800288018120843194988421FD194F823020106F1
S3150800289094F8220241EA004194F8210241EA002014
S315080028A094F820120843E06094F81F02010600E03D
S315080028B00BE094F81E0241EA004194F81D0241EA31
S315080028C0002094F81C1208432061257008480088E7
S315080028D0401C80B206490880E080002020632071F1
S315080028E000BF59E6340000205252614172724161BC
S315080028F0380000200246891E9069801E884201D849
S31508002900002070479378D06A01FB0300F9E70000BE
S315080029102DE9F04705460C46207820F04000401E79
S3150800292000EB800101EBC00600274FF0010800BF4D
S315080029301A48C05D205C1949C95D2144497840EAB6
S315080029400129B8F1000F10D0484601F0ADFB8046CA
S31508002950FF2E07D23146761C35F8110001F0A4FB8C
S31508002960404508D00020BDE8F0874FF6FF70814546
S3150800297001D00020F7E7781C07460D28D8D3207821
S3150800298000F0400038B1B8F1000F04D035F8160051
S3150800299008B10020E7E70120E5E70000704D0008D0
S315080029A02DE9F04704468946B9F1000F06D1E768D4
S315080029B017B1A069B84211D801270FE04946204649
S315080029C001F06BFC0646022E02D20120BDE8F08714
S315080029D0A069B04201D93046F8E74F463D4600BFE8
S315080029E06D1CA069A84204D80225BD4201D9002061
S315080029F0ECE72946204601F050FC064606B909E0F0
S31508002A00701C08B1012E01D13046DFE7BD42E7D17F
S31508002A100020DBE700BF6FF070422946204601F030
S31508002A204DFE8046B8F1000F08D1B9F1000F05D068
S31508002A302A464946204601F041FE8046B8F1000F75
S31508002A4009D1E5602069401C68B12069401E2061F3
S31508002A500120607107E0B8F1010F02D14FF0FF3095
S31508002A6000E0012005462846B0E700002DE9F34FAF
S31508002A7083B08246002000900498D0F800B001E0A8
S31508002A800BF1010B9BF800002F28F9D09BF80000EA
S31508002A905C28F5D0DAF81C9000252E4600BF304693
S31508002AA0761C1BF80040202C03DB2F2C01D05C2C55
S31508002AB000D11CE0FF2D03D3062005B0BDE8F08F3A
S31508002AC0E4B20121204601F0C9FA04460CB90620F1
S31508002AD0F3E7802C06DA21466BA0FFF733FD08B131
S31508002AE00620EAE728466D1C29F81040D7E700BFFC
S31508002AF00BEB060104980160202C01DA042000E0A3
S31508002B000020074608E0681E39F81040202C02D03D
S31508002B102E2C00D002E06D1E002DF4D100BF0DB999
S31508002B200620CAE7002029F815000B222021DAF82A
S31508002B30180001F0F5FC002600E0761C39F81600AE
S31508002B402028FAD039F816002E28F6D00EB147F00C
S31508002B50030700E06D1E25B1681E39F810002E28FF
S31508002B60F8D14FF00008CDF808800820019000BF82
S31508002B703046761C39F8104004B955E0202C03D0AD
S31508002B802E2C04D1AE4202D047F00307F0E7DDE968
S31508002B900110884201D2AE4216D101980B2802D103
S31508002BA047F0030740E0AE4201D047F00307AE42C4
S31508002BB000D939E02E46082002900B2001904FEAF2
S31508002BC088604FEA1068D3E7802C0BDB002120468B
S31508002BD001F044FA04461CB1A4F180002D490C5CAE
S31508002BE047F0020700BF24B121462BA0FFF7AAFC35
S31508002BF018B15F2447F003070FE0412C04DB5A2C79
S31508002C0002DC48F0020808E0612C06DB7A2C04DCBA
S31508002C1048F00108A4F1200084B2DAF818300298C6
S31508002C20411C02911C54A3E700BFDAF8180000788B
S31508002C30E52803D10520DAF8181008700198082845
S31508002C4003D14FEA88604FEA106808F00C000C2898
S31508002C5003D008F00300032801D147F0020707F064
S31508002C60020058B908F00300012801D147F01007FF
S31508002C7008F00C00042801D147F00807DAF8180014
S31508002C80C772002019E70000222A3A3C3E3F7C7FA3
S31508002C9000000000F04C00082B2C3B3D5B5D00005B
S31508002CA010B54FF480510348FEF724FEFF2001F0CB
S31508002CB0B1FF10BD000C01402DE9F04104460E4657
S31508002CC00021204600F049FA0546EDB9002700BF65
S31508002CD02169206801F02EFC054605B113E06069FC
S31508002CE00078E52802D06069007820B9781C074684
S31508002CF0B04201D107E000270121204600F076F80E
S31508002D000546002DE4D000BF2846BDE8F0812DE930
S31508002D10F04704460021204600F01FFA074617B17F
S31508002D203846BDE8F0874FF0FF09CA4600BF21695B
S31508002D30206801F0FFFB074607B154E065692E7865
S31508002D400EB904274FE0E87A00F03F08E52E05D0D3
S31508002D5008F0080028B1B8F10F0F02D04FF0FF09AC
S31508002D603AE0B8F10F0F1CD1E069A0B306F04000B5
S31508002D7030B195F80DA026F04006B146E0882084CB
S31508002D804E450AD1687B504507D12946E069FFF7C9
S31508002D90BFFD10B1A9F1010000E0FF2000F0FF0916
S31508002DA01AE0B9F1000F05D1284601F065FE504535
S31508002DB000D118E04FF0FF094FF6FF702084A06994
S31508002DC0C07A00F0010030B90B222846A16901F04B
S31508002DD087FB00B907E0FFE70021204600F006F868
S31508002DE00746002FA3D000BF38469AE72DE9F041E1
S31508002DF00446884600BFE088401C86B20EB12069AA
S31508002E0010B90420BDE8F08106F00F0000286DD146
S31508002E102069401C2061E06828B920680089B04212
S31508002E2064DC0420EEE720688078401E00EA16106D
S31508002E3000285BD1E168206801F02FFA0546012DCC
S31508002E4001D80220DEE7681C08B90120DAE7206805
S31508002E508069A84244D8B8F1000F01D10420D1E70F
S31508002E60E1682068FFF79CFD05460DB90720C9E70C
S31508002E70012D01D10220C5E7681C08B90120C1E768
S31508002E80206801F06DFE08B10120BBE7216801F159
S31508002E9034004FF40072002101F042FB29462068F5
S31508002EA0FFF728FD2168086300270FE00120216845
S31508002EB00871206801F054FE08B10120A2E72068D5
S31508002EC0006B401C21680863781CC7B220688078AC
S31508002ED0B842EBDC2068006BC01B2168086300BFA2
S31508002EE0E56029462068FFF705FD2061E680206831
S31508002EF0343006F00F0100EB41106061002081E7D5
S31508002F002DE9F05F04468A464FF0FF09CB460427B1
S31508002F104EE02169206801F00DFB074607B14AE03B
S31508002F20666935780DB9042745E0F07A00F03F0860
S31508002F30E52D09D02E2D07D0B8F1080F01D10120B3
S31508002F4000E00020504502D04FF0FF0929E0B8F113
S31508002F500F0F1AD105F0400030B196F80DB025F0E4
S31508002F604005A946E08820844D450AD1707B58451E
S31508002F7007D13146E06901F0F7FA10B1A9F101006D
S31508002F8000E0FF2000F0FF090BE0B9F1000F04D1C3
S31508002F90304601F071FD584502D04FF6FF70208487
S31508002FA009E000212046FFF721FF074607B102E0A6
S31508002FB020690028ADD100BF0FB100202061384636
S31508002FC0BDE8F09F2DE9FE4F0446D4F81880D4F8E2
S31508002FD01C900C224146684601F095FA00BF9DF800
S31508002FE00B0000F0010028B3002088F80B00E06110
S31508002FF001260DE033464A466946404601F0F9F88F
S315080030002046FFF784FE054605B103E0701C86B22C
S31508003010642EEFDB00BF642E02D10720BDE8FE8FC9
S31508003020042D01D02846F9E79DF80B0088F80B0017
S31508003030C4F81C909DF80B0000F0020070B1002641
S3150800304001E0701C86B239F816000028F9D106F19D
S3150800305019000D2190FBF1F087B200E001273946EF
S315080030602046FFF729FE05465DBB781E80B2071E7F
S3150800307027D0E088C01B81B2204600F06EF80546CE
S31508003080FDB9A06901F0F8FC824600BF21692068F5
S3150800309001F050FA054605B112E0FAB253466169E5
S315080030A0E06901F01DF80120216808710021204619
S315080030B0FFF79CFE05461DB9781E80B2071EE5D1AE
S315080030C000BFC5B92169206801F034FA054695B9EB
S315080030D020220021606901F023FA0B22D4E90501B8
S315080030E001F011FAA069C07A00F018006169087346
S315080030F0012021680871284690E770B50446E688DD
S31508003100208C4FF6FF72904201D1304600E0208CA9
S315080031100146204600F021F80546E5B900BF2169B9
S31508003120206801F007FA054605B110E0E520616957
S315080031300870012021680871E088B04200DB06E0CB
S3150800314000212046FFF752FE0546002DE7D000BFB6
S31508003150042D00D10225284670BD2DE9F04104460C
S315080031600E46E680A568012D03D020688069A8422E
S3150800317002D80220BDE8F0812DB92068007803281E
S3150800318001D12068856A65B9E56020680089B04282
S3150800319001DC0220EEE72068806A00EB1610206149
S315080031A020E020688078070112E02946206801F0AF
S315080031B074F80546681C08B90120DBE7022D03D31D
S315080031C020688069A84201D80220D3E7F01B86B29E
S315080031D0BE42EADAE56029462068FFF78BFB00EB7A
S315080031E0161020612068343006F00F0100EB4110FC
S315080031F060610020BEE700002DE9F8438046B8F17B
S31508003200000F02D00120BDE8F8834948007800F095
S31508003210020010B146480078F5E701F0E9F94FF4E5
S3150800322080514448FEF764FB00270021084601F058
S315080032305BFB012868D1FEF763FD00F57A754FF44C
S31508003240D571082001F050FB01283CD1002406E086
S31508003250FF2001F0DFFC0DF80400601CC4B2042C4A
S31508003260F6DB9DF8020001284ED19DF80300AA2836
S315080032704AD100BFFEF744FDA84206D24FF080416E
S31508003280A92001F031FB0028F4D1FEF739FDA84248
S315080032903AD200213A2001F027FBA8BB002406E019
S315080032A0FF2001F0B7FC0DF80400601CC4B2042C22
S315080032B0F6DB9DF8000000F0400008B10C2000E0A5
S315080032C00420074620E00021A92001F00DFB012873
S315080032D002DC0227A92601E00127012600BFFEF726
S315080032E00FFDA84205D20021304601F0FDFA00285C
S315080032F0F5D1FEF705FDA84205D24FF4007110205E
S3150800330001F0F2FA00B100270B480760FFF7C8FC86
S3150800331047B10748007820F001000549087001F018
S3150800332071FB01E001F05AF9014800786BE70000EB
S3150800333014000020000C0140180000202DE9FF476A
S3150800334080460F461446A246B8F1000F03D0042063
S3150800335004B0BDE8F0878548007800F0010008B1A0
S315080033600320F5E74FF001090F2F7AD2DFE807F0BF
S31508003370080EF655F6F6F6F6F6F6AEB5C2CFE10045
S3150800338001F09EFA08B14FF00009EAE00021092091
S3150800339001F0AAFAE8BB1021684601F02AFAC0B380
S315080033A09DF800000121B1EBA01F0FD19DF809007F
S315080033B09DF8081000EB01209DF8071001F03F0169
S315080033C000EB0140461CB002206021E09DF8050094
S315080033D000F00F009DF80A1000EBD1109DF80910B7
S315080033E001F0030100EB4100851C9DF808008011DF
S315080033F09DF8071000EB81009DF8061001F0030107
S3150800340000EB8120461CA5F1090006FA00F02060B1
S3150800341000E001E04FF00009A3E05548007800F00D
S315080034200400F8B100218D2001F05EFA00284CD185
S31508003430FF2001F0EFFB1021684601F0DAF988B3A6
S31508003440302504E0FF2001F0E5FB681EC5B2002D1B
S31508003450F8D19DF80A000111102088402060A9467D
S3150800346033E07BE00021092001F03EFAD0B91021B3
S31508003470684601F0BEF9A8B13D48007800F00200A0
S3150800348088B19DF80A008006400E9DF80B1000EBE7
S31508003490D110401C9DF80D100122C2EBA1118840E5
S315080034A0206010E011E09DF80B008007C00E9DF823
S315080034B00B1000EB5110401C9DF80A10C1F3840153
S315080034C0491C484320604FF000094AE02848007824
S315080034D08AF800004FF0000943E00021092001F0B6
S315080034E003FA30B91021204601F083F908B14FF0EC
S315080034F0000936E000210A2001F0F6F930B910215A
S31508003500204601F076F908B14FF0000929E00021BC
S315080035103A2001F0E9F958B9002505E0FF2001F045
S3150800352079FB6055681CC5B2042DF7DB4FF000091E
S3150800353017E00F48007800F0040070B100218D20D4
S3150800354001F0D2F948B9FF2001F064FB402120467A
S3150800355001F04FF908B14FF0000902E04FF00409F5
S3150800356000BF00BFFFF79CFB4846F1E614000020A9
S31508003570180000202DE9F04107460D4616461C4660
S3150800358007B914B90420BDE8F0811D48007800F099
S31508003590010008B10320F6E71A48007800F0080091
S315080035A000B97602012C0BD13146112001F09CF9A5
S315080035B0F0B96102284601F01CF9C8B1002417E0E9
S315080035C03146122001F090F990B900BF4FF400710E
S315080035D0284601F00EF900B905E005F50075601EEC
S315080035E0C0B2041EF2D100BF00210C2001F07CF904
S315080035F0FFF756FB0CB10120C5E70020C3E7000022
S315080036001400002018000020014609B10120704767
S3150800361001480078FBE70000140000202DE9F0417E
S3150800362007460D4616461C4607B914B90420BDE8D8
S31508003630F0812548007800F0010008B10320F6E77C
S315080036402148007800F0040008B10220EFE71F487F
S31508003650007800F0080000B97602012C0BD131463B
S31508003660182001F041F940BBFE21284601F0E6FA90
S3150800367018B3002421E01548007800F0060018B1B8
S315080036802146972001F030F93146192001F02CF92E
S3150800369098B900BFFC21284601F0D0FA00B905E028
S315080036A005F50075601EC0B2041EF3D100BFFD21EA
S315080036B0002001F0C3FA00B90124FFF7F1FA0CB1B2
S315080036C00120B4E70020B2E714000020180000200B
S315080036D070B50446204600F009FB05460DB90020E2
S315080036E02060284670BD2DE9FC4707468846914666
S315080036F000253E4615E06B46012201A9484600F022
S31508003700EDF90098012800D00FE09DF804400D2C33
S3150800371000D106E006F8014B6D1C0A2C00D104E026
S3150800372000BFA8F10100A842E5DC00BF0020307008
S3150800373015B13846BDE8FC870020FBE72DE9F047C0
S3150800374004460E46204601F034FA8246BAF1000FC6
S3150800375002D05046BDE8F087A07900F0800008B195
S315080037600220F7E7E068B04204D2A07900F0020030
S3150800377000B9E668D4F808904FF00008C4F8088045
S31508003780002E77D0206880784702B9F1000F11D053
S31508003790701EB0FBF7F1A9F10100B0FBF7F081420A
S315080037A008D3A9F10100791E8843A060A068361ADB
S315080037B0656918E02569ADB900212068FFF7F0F8BA
S315080037C00546012D05D1A07940F08000A0710220A0
S315080037D0C0E7681C28B9A07940F08000A0710120D4
S315080037E0B8E725616561002D44D029E0A07900F08D
S315080037F0020038B129462068FFF7D2F8054635B9E0
S315080038003E461FE02946206800F047FD0546681C2D
S3150800381028B9A07940F08000A07101209AE7012D0F
S3150800382003D920688069A84205D8A07940F08000AD
S31508003830A07102208EE76561A0683844A060F61B77
S31508003840BE42D3D800BFA0683044A060C6F30800C3
S3150800385068B129462068FFF74DF88046B8F1000F91
S3150800386006D1A07940F08000A071022072E701E03D
S3150800387008EB56282089C0F3080050B3A0694045D4
S3150800388027D0A07900F0400090B12168487801233C
S3150800389004F12401A269FFF7C1FE28B1A07940F01E
S315080038A08000A071012055E7A07920F04000A071A2
S315080038B0216848780123424604F12401FFF75AFE9D
S315080038C028B1A07940F08000A071012042E7C4F831
S315080038D01880D4E90201884205D9A068E060A07979
S315080038E040F02000A071504634E700000246012A45
S315080038F001DB0B207047074850F822300BB1002037
S31508003900187009B100200870024840F822100020FB
S31508003910F0E70000340000202DE9F7438CB0054697
S3150800392016461DB909200FB0BDE8F08300202860AF
S3150800393006F01F0626F0010203A90DA8FEF70CFEE5
S315080039400746002F7ED1CDF824D04C480A9003A80C
S315080039500D9900F005FC0746089C0FB904B906271F
S3150800396006F01C00002851D04FB1042F03D103A83C
S31508003970FFF728FB074646F00806089C09E0E07AA8
S3150800398000F0110008B1072703E006F0040000B1B3
S315080039900827002F39D106F00800002835D000F096
S315080039A0EFFC804684F80E804FEA1821E1734FEA4F
S315080039B0184121744FEA186161740020E07220777B
S315080039C000216177A177E1772146039800F070FD21
S315080039D081460021204601F047F801200399087125
S315080039E0B9F1000F11D00398D0F8308049460398F2
S315080039F000F032FF074647B9A9F101000399C860EC
S31508003A004146039800F096FD07460EE06FB9E07A46
S31508003A1000F0100008B1042707E006F0020020B104
S31508003A20E07A00F0010000B1072747B906F0080060
S31508003A3008B146F020060398006BE8612C620FB9BE
S31508003A40AE7100E017E02146039800F031FD2861C9
S31508003A50E07F0106A07F41EA0041607F41EA00203D
S31508003A60217F0843E8600020A860A86103982860C1
S31508003A700398C088A880384655E700001809002032
S31508003A807CB504460E460A2C03D131460D20FFF7B5
S31508003A90F7FF8DF80040012501AB2A4669463046F6
S31508003AA000F0D6F90198A84200D17CBD4FF0FF304E
S31508003AB0FBE770B504460E4600250AE02078314635
S31508003AC0FFF7DEFF401C10B94FF0FF3070BD641CD5
S31508003AD06D1C20780028F1D12846F7E72DE9FF4F1D
S31508003AE083B0044615469A46DDF810B00020CAF899
S31508003AF00000204601F05DF80290029818B102987D
S31508003B0007B0BDE8F08FA07900F0800008B1022068
S31508003B10F6E7A07900F0010008B90720F0E7D4E934
S31508003B200210401A00900098854200D9009DB5E021
S31508003B302089C0F3080000287ED120688078401EBE
S31508003B40A16800EA512000F0FF09B9F1000F1DD164
S31508003B50A06810B92069019004E06169206800F046
S31508003B609CFB01900198022805D2A07940F08000BC
S31508003B70A0710220C4E70198401C28B9A07940F03A
S31508003B808000A0710120BBE7019860616169206827
S31508003B90FEF7B0FE06462EB9A07940F08000A07167
S31508003BA00220ADE74E444FEA5528B8F1000F2DD054
S31508003BB009EB080021688978884203D9206880784B
S31508003BC0A0EB090808F0FF032168487832465946F1
S31508003BD0FFF7D0FC28B1A07940F08000A071012041
S31508003BE08EE7A07900F0400068B1A069801B4045C7
S31508003BF009D2A169891B0BEB41204FF4007204F12D
S31508003C00240100F080FC4FEA48273DE0A069B04255
S31508003C1026D0A07900F0400098B1216848780123A1
S31508003C2004F12401A269FFF7F9FC30B1A07940F04C
S31508003C308000A071012063E713E0A07920F040001E
S31508003C40A071216848780123324604F12401FFF760
S31508003C5091FC28B1A07940F08000A07101204FE7BF
S31508003C60A6612089C0F30800C0F50077AF4200D9E5
S31508003C702F462089C0F3080204F1240011183A4699
S31508003C80584600F040FC00BFBB44A0683844A0601A
S31508003C90DAF800003844CAF80000ED1B002D7FF45E
S31508003CA047AF00202CE7000033B58DB00D46002243
S31508003CB004A90DA8FEF750FC04468CB901A80A9081
S31508003CC009480B9004A80D9900F04AFA04463CB935
S31508003CD0099820B1294604A800F056FB00E00624FE
S31508003CE020460FB030BD0000180900202DE9F0412C
S31508003CF00446204600F05DFF0746002F4CD1A07908
S31508003D0000F02000002847D0A07900F0400078B1E4
S31508003D1021684878012304F12401A269FFF77EFC93
S31508003D2010B10120BDE8F081A07920F04000A07113
S31508003D30E169206800F0FEFB0746002F2CD1256AB2
S31508003D40E87A40F02000E872207B2877A089010AEB
S31508003D506977E068010CA977E068010EE9772846DB
S31508003D60216900F081FE00F00BFB0646AE75310AAC
S31508003D70E975310C2976310E69760020A874002180
S31508003D80E974A07920F02000A0710120216808714B
S31508003D90206800F081FE07463846C3E771B595B03E
S31508003DA001220CA915A8FEF7D7FB0446002C49D119
S31508003DB0CDF848D0254813900CA8159900F0D0F9ED
S31508003DC0044600BF002C3DD1119E0EB9062404E01E
S31508003DD0F07A00F0010000B1072431460C9800F093
S31508003DE067FB0546ECB9F07A00F01000C8B1022D61
S31508003DF001D2022415E024220CA903A800F083FBB3
S31508003E000595022103A8FFF7A8F904464CB9002135
S31508003E1003A8FFF775F8044604B90724042C00D153
S31508003E2000247CB90CA8FFF768F9044654B925B1F3
S31508003E3029460C9800F010FD04461CB90C9800F0B1
S31508003E402BFE0446204616B070BD00001809002057
S31508003E502DE9FF4F83B0044615469B46049801900A
S31508003E600020CBF80000204600F0A3FE029002983E
S31508003E7018B1029807B0BDE8F08FA07900F080006D
S31508003E8008B10220F6E7A07900F0020008B9072079
S31508003E90F0E7E0682844E168884200D20025CDE0D2
S31508003EA02089C0F30800002877D120688078401E52
S31508003EB0A16800EA512000F0FF0ABAF1000F2AD1E2
S31508003EC0A06858B9D4F81080B8F1000F0BD10021BA
S31508003ED02068FEF765FD8046206104E06169206878
S31508003EE0FEF75EFD8046B8F1000F00D1A9E0B8F1F3
S31508003EF0010F05D1A07940F08000A0710220B9E732
S31508003F0008F1010028B9A07940F08000A0710120CD
S31508003F10B0E7C4F81480A07900F0400090B1216899
S31508003F204878012304F12401A269FFF777FB28B139
S31508003F30A07940F08000A07101209BE7A07920F0CD
S31508003F404000A07161692068FEF7D4FC06462EB9C8
S31508003F50A07940F08000A07102208BE756444FEA12
S31508003F605529B9F1000F2FD00AEB09002168897885
S31508003F70884203D920688078A0EB0A0909F0FF0374
S31508003F802168487832460199FFF748FB30B1A07995
S31508003F9040F08000A07101206CE72CE0A069801B2E
S31508003FA048450ED2A069801B019A02EB40214FF4C6
S31508003FB0007204F1240000F0A6FAA07920F040006F
S31508003FC0A0714FEA49272DE0A069B04212D0D4E982
S31508003FD0020188420ED2216848780123324604F14C
S31508003FE02401FFF7C7FA28B1A07940F08000A07134
S31508003FF001203FE7A6612089C0F30800C0F50077D5
S31508004000AF4200D92F462189C1F3080204F12401E1
S3150800401050183A46019900F076FAA07940F0400027
S31508004020A07100BF019838440190A0683844A06088
S31508004030DBF800003844CBF80000ED1B002D7FF4B8
S315080040402FAF00BFD4E90201884201D9A068E06019
S31508004050A07940F02000A07100200BE710B50246B9
S31508004060802A01DA10461BE051B1FF2A01DD002340
S3150800407004E0A2F180030B4C34F8133018460FE025
S31508004080002007E0074B33F81030934200D103E0D5
S31508004090431C98B28028F5DB00BF00F18003D8B234
S315080040A010BD00007E4D00080246002100E0491CB4
S315080040B0094830F8110020B1074830F8110090423D
S315080040C0F5D1054830F8110018B1044830F8110048
S315080040D070471046FCE700007E4E00085E50000858
S315080040E0F0B504461D464D730F27CF7200270F7390
S315080040F08F76BC4681F81BC0571E07EB870C0CEB66
S31508004100C706002738463B4600BF4FF6FF77B8423A
S3150800411003D03746761C34F81700DFF840C01CF881
S3150800412003C001F80C000712DFF830C01CF803C002
S315080041308C448CF8017008B94FF6FF705F1C3B463B
S315080041400D2FE2D34FF6FF77B84202D034F8167037
S315080041500FB942F040020A70F0BD0000704D000829
S315080041602DE9F3410446019800782F2803D00198D9
S3150800417000785C2802D10198401C01900020A060BC
S3150800418001980078202807D200212046FEF7E5FF8F
S3150800419005460020606129E000BF01A92046FEF718
S315080041A065FC054605B120E02046FEF7B0FD05464C
S315080041B0A069C67A45B1042D00D016E000BF06F006
S315080041C0040000B9052510E006F0040000B10CE073
S315080041D06769F87A00F0100008B9052505E0394640
S315080041E0206800F065F9A060D7E700BF2846BDE85B
S315080041F0FC812DE9FC4780468A4617461C460B2259
S315080042005146404600F07FF9052C0ADD00BF6010D4
S3150800421000EBC43137F8022B881884B23888002896
S31508004220F5D1072500BF2046E11704EB11710911E6
S31508004230A4EB0111303101F0FF09B9F1390F03DDA3
S3150800424009F1070000F0FF0928466D1E0DF80090D9
S315080042502046E11704EB1171C1F30F14002CE2D1CB
S315080042607E200DF80500002600E0761CAE4203D23B
S3150800427018F806002028F8D100BF082D04D22846D1
S315080042806D1C1DF8000000E020203146761C08F859
S315080042900100082EF1D3BDE8FC872DE9F04105465B
S315080042A00C46022C02D3A869A04202D80120BDE818
S315080042B0F0812878012804D002282CD003285AD166
S315080042C03DE0274607EB5707686A00EB5721284663
S315080042D000F030F900B14EE0C7F3080105F13400EB
S315080042E010F801807F1C686A00EB5721284600F009
S315080042F021F900B13FE0C7F3080105F13400405C3D
S3150800430048EA002804F0010010B14FEA1810CEE779
S31508004310C8F30B00CBE7686A00EB1421284600F0C7
S3150800432009F900B127E040F2FF1000EA440105F15F
S3150800433034000E183078717840EA0120B7E7686AC9
S3150800434000EBD411284600F0F5F800B113E040F26E
S31508004350FF1000EA840105F134000E18F078000613
S31508004360B17840EA0140717840EA01203178084383
S3150800437020F070409BE700BF4FF0FF3097E7000042
S31508004380004870470000AA422DE9FC5F81460E46A8
S3150800439006F10908D9F81000002851D0D9F81440B8
S315080043A0207B0190002714E0E55D202D00D112E066
S315080043B0052D00D1E525019800F0080030B1412D02
S315080043C004DB5A2D02DC05F12000C5B208F8015BB2
S315080043D07F1C082FE8D300BF207A202819D02E206A
S315080043E008F8010B082711E0E55D202D00D10FE044
S315080043F0019800F0100030B1412D04DB5A2D02DC83
S3150800440005F12000C5B208F8015B7F1C0B2FEBD322
S3150800441000BFE07A3072E07F0106A07F41EA0041E2
S31508004420607F41EA0020217F08433060217E607E5C
S3150800443041EA0020B080A17DE07D41EA0020F080BD
S31508004440002088F80000B06980B3F06970B3B069DD
S3150800445000900027D9F8100020B3B9F820004FF6CD
S31508004460FF7188421ED0D9F81CB015E000215046CD
S31508004470FFF7F4FD8246BAF1000F01D1002710E0DC
S3150800448000BFF069401EB84201D8002709E0384647
S315080044907F1C009901F800A03BF8021BB1F1000A45
S315080044A0E4D100BF00210098C15500BFBDE8FC9FBC
S315080044B010B502468C7ECB7E44EA03201378032B84
S315080044C005D10C7D4B7D44EA032340EA034010BD29
S315080044D0FDF712FAFBF77CFF01E0FBF789FFFCE723
S315080044E0F0B503461C460D46002000BF161EA2F175
S315080044F0010207D014F8017B15F801CBA7EB0C06CF
S31508004500301EF3D0F0BD70B503460C4603E014F830
S31508004510015B03F8015B151EA2F10102F7D170BD1C
S3150800452030B5034601E003F8011B141EA2F101028F
S31508004530F9D130BD70B504460D46206BA84210D09F
S31508004540204600F00DFB08B1012070BD60780123FC
S315080045502A4604F13401FFF70DF808B10120F4E703
S3150800456025630020F1E70000F0B50346087800F05F
S315080045703F00401E00EB800707EBC002002501261E
S3150800458000BF1548405D085C134F7F5D0F447F7878
S3150800459040EA07244EB1FF2A01D30020F0BD264683
S315080045A01046521C23F8104005E04FF6FF7084426F
S315080045B001D00020F2E7681C05460D28E1D30878EB
S315080045C000F0400030B1FF2A01D30020E6E70020C2
S315080045D023F812000120E1E7704D0008034800782F
S315080045E040F00100014908707047000014000020DF
S315080045F000B587B001210820FDF720FA01218803BC
S31508004600FDF70CFA4FF48050ADF8040010208DF831
S31508004610070003208DF8060001A92648FDF794F83F
S315080046204FF480512348FDF765F94FF42040ADF863
S31508004630040003208DF8060018208DF8070001A94C
S315080046401C48FDF781F84FF48040ADF80400482077
S315080046508DF8070001A91748FDF776F80020ADF890
S3150800466008004FF48270ADF80A000020ADF80C007F
S31508004670ADF80E00ADF810004FF40070ADF812005A
S315080046803820ADF814000020ADF816000720ADF864
S31508004690180002A90848FDF771FA00210648FDF737
S315080046A047FA01210448FDF74FFA00F067F907B009
S315080046B000BD0000000C0140003800402DE9F0471D
S315080046C005460E461746022E02D3A869B04202D8FE
S315080046D04FF002088AE02878012804D0022841D041
S315080046E003287DD154E0B14609EB5909686A00EB05
S315080046F059212846FFF71EFF8046B8F1000F00D063
S3150800470071E0C9F3080105F134000C1806F0010040
S3150800471020B1F9B2207861F31F1000E03846207006
S3150800472009F1010901202871686A00EB5921284618
S31508004730FFF700FF8046B8F1000F00D053E0C9F339
S31508004740080105F134000C1806F0010010B1C7F392
S31508004750071005E0207800F0F000C7F303210843AE
S31508004760207040E0686A00EB16212846FFF7E2FE53
S315080047708046B8F1000F00D035E040F2FF1000EA9D
S31508004780460105F134000C182770380A60702AE0D3
S31508004790686A00EBD6112846FFF7CCFE8046B8F1CA
S315080047A0000F00D01FE040F2FF1000EA860105F175
S315080047B034000C18E0780006A17840EA01406178D8
S315080047C040EA01202178084300F07040074327702B
S315080047D0380A6070380CA070380EE07003E0FFE706
S315080047E04FF0020800BF00BF012028714046BDE80F
S315080047F0F0872DE9F04105460E46FDF781FA00F1EE
S31508004800640700BFFF2000F005FA0446FF2C03D119
S31508004810FDF776FAB842F5D3FE2C02D00020BDE8A3
S31508004820F08100BF28466D1C00F00FF828466D1C65
S3150800483000F00BF8B01E061EF4D1FF2000F0EAF9CE
S31508004840FF2000F0E7F90120E9E710B50446FF204C
S3150800485000F0E0F9207010BD2DE9F04104460E463F
S31508004860022E02D3A069B04201D8022725E000270C
S315080048701FE031462046FFF710FD054605B91BE047
S31508004880012D01D1022717E0681C08B9012713E09A
S31508004890002231462046FFF711FF074607B10BE015
S315080048A02069401C20B12069401C206101206071EC
S315080048B02E46A069B042DCD800BF3846BDE8F08174
S315080048C010B54FF480510748FDF712F8FF2000F0A5
S315080048D0A1F900F089F908B1012010BDFEF7E0F949
S315080048E00020FAE7000C01402DE9F04104460D4688
S315080048F004F0800058B104F07F0400213720FFF748
S31508004900F3FF0646012E02DD3046BDE8F081FEF7CC
S31508004910C7F9FFF7D5FF08B9FF20F6E744F04000CE
S3150800492000F078F9280E00F075F9C5F3074000F095
S3150800493071F9C5F3072000F06DF9E8B200F06AF9DD
S31508004940012704B99527082C00D18727384600F097
S3150800495061F90C2C02D1FF2000F05CF90A2700BF90
S31508004960FF2000F057F9064606F0800018B1781EB9
S31508004970C0B2071EF4D13046C7E7000038B54FF479
S3150800498080511E48FCF7B6FF4FF40040ADF8000012
S3150800499003208DF8020010208DF803006946174899
S315080049A0FCF7D2FE4FF400411448FCF7A3FF00249D
S315080049B012E000BF02211248FDF7D2F80028F9D00C
S315080049C0FF210F48FDF7D8F800BF01210C48FDF775
S315080049D0C7F80028F9D0641C0A2CEAD34FF4004023
S315080049E0ADF8000003208DF8020018208DF80300AA
S315080049F069460248FCF7A8FE38BD0000000C0140D5
S31508004A000038004000B585B000211648FDF79CF82F
S31508004A100020ADF800004FF48270ADF802000020C7
S31508004A20ADF80400ADF80600ADF808004FF40070C4
S31508004A30ADF80A000820ADF80C000020ADF80E000D
S31508004A400720ADF8100069460648FDF797F80021DB
S31508004A500448FDF76DF801210248FDF775F805B021
S31508004A6000BD00000038004081760B0AC3760A0CA8
S31508004A7002750B0E4375704730B5014600200B22B0
S31508004A8000BF431003EBC01411F8015B6319D8B2D9
S31508004A90531E1A1EF5D130BD70B50446204600F0E7
S31508004AA05FF80546002D59D1207803284FD1607943
S31508004AB000284CD0002020634FF40072002104F136
S31508004AC03400FFF72DFD552184F83212AA2184F807
S31508004AD03312522084F834005221352001556121C1
S31508004AE036200155412137200155722184F81812C4
S31508004AF084F81912412184F81A12612184F81B12CC
S31508004B00217C84F81C12208A010A84F81D12206967
S31508004B10010C84F81E122069010E84F81F12217BED
S31508004B2084F82012A089010A84F82112E068010C91
S31508004B3084F82212E068010E84F8231260780123B3
S31508004B4004F134016269FEF769FD0020607160783E
S31508004B5000221146FEF7F2FB00B10125284670BD7A
S31508004B6070B50446207910B3256B607801232A4670
S31508004B7004F13401FEF752FD08B1012070BD002092
S31508004B802071606AA84212D8E169606A0844A8429E
S31508004B900DD9E67809E0E0690544607801232A46DC
S31508004BA004F13401FEF73AFD761E022EF3D20020F8
S31508004BB0E4E770B505462C464CB1206838B1206844
S31508004BC0007820B12068C088A188884201D00920D1
S31508004BD070BD21684878FEF717FD00F0010008B19E
S31508004BE00320F5E70020F3E770B5FDF789F800F52F
S31508004BF0FA7500BFFF2000F00DF80446FF2C03D01D
S31508004C00FDF77EF8A842F5D3FF2C01D1012070BD2F
S31508004C100020FCE710B5044621460748FCF7ACFF20
S31508004C2000BF01210448FCF79BFF0028F9D0024881
S31508004C30FCF79FFFC0B210BD003800402DE9F041D7
S31508004C4004460D46FFF7D0FF10B90020BDE8F081F5
S31508004C502846FFF7DFFFFD2D1DD04FF4007700BF74
S31508004C6014F8010BFFF7D6FF14F8010BFFF7D2FF74
S31508004C70B81E071EF4D1FF20FFF7CCFFFF20FFF771
S31508004C80C9FFFF20FFF7C6FF064606F01F000528E6
S31508004C9001D00020DAE70120D8E7000010B5002986
S31508004CA00AD00878002807D005487844FBF7E2FAC6
S31508004CB0002801D0002010BD0248784410BD00002D
S31508004CC0760600006E0600002F64656D6F70726FC1
S31508004CD0675F6F6C696D65785F73746D33327031B9
S31508004CE030332E73726563004F70656E424C540004
S31508004CF0809A90418E418F804545454949498E8F16
S31508004D009092924F994F555559999A9B9C9D9E9F63
S31508004D1041494F55A5A5A6A7A8A9AAABAC21AEAFF0
S31508004D20B0B1B2B3B4B5B6B7B8B9BABBBCBDBEBFFD
S31508004D30C0C1C2C3C4C5C6C7C8C9CACBCCCDCECFED
S31508004D40D0D1D2D3D4D5D6D7D8D9DADBDCDDDEDFDD
S31508004D50E0E1E2E3E4E5E6E7E8E9EAEBECEDEEEFCD
S31508004D60F0F1F2F3F4F5F6F7F8F9FAFBFCFDFEFFBD
S31508004D7001030507090E10121416181C1E00C70099
S31508004D80FC00E900E200E400E000E500E700EA00D4
S31508004D90EB00E800EF00EE00EC00C400C500C90017
S31508004DA0E600C600F400F600F200FB00F900FF007A
S31508004DB0D600DC00A200A300A500A7209201E1000E
S31508004DC0ED00F300FA00F100D100AA00BA00BF0016
S31508004DD01023AC00BD00BC00A100AB00BB009125B0
S31508004DE092259325022524256125622556255525D4
S31508004DF06325512557255D255C255B25102514253A
S31508004E0034252C251C2500253C255E255F255A259D
S31508004E10542569256625602550256C25672568254E
S31508004E206425652559255825522553256B256A2558
S31508004E3018250C25882584258C2590258025B103E1
S31508004E40DF009303C003A303C303B500C403A6038B
S31508004E509803A903B4031E22C603B50329226122B7
S31508004E60B1006522642220232123F7004822B000DE
S31508004E701922B7001A227F20B200A025A0006100DF
S31508004E8062006300640065006600670068006900E8
S31508004E906A006B006C006D006E006F007000710098
S31508004EA07200730074007500760077007800790048
S31508004EB07A00A100A200A300A500AC00AF00E000A4
S31508004EC0E100E200E300E400E500E600E700E800B0
S31508004ED0E900EA00EB00EC00ED00EE00EF00F00060
S31508004EE0F100F200F300F400F500F600F800F9000E
S31508004EF0FA00FB00FC00FD00FE00FF0001010301B3
S31508004F000501070109010B010D010F01110113012B
S31508004F101501170119011B011D011F01210123019B
S31508004F202501270129012B012D012F01310133010B
S31508004F30350137013A013C013E0140014201440175
S31508004F40460148014B014D014F01510153015501DD
S31508004F50570159015B015D015F016101630165014B
S31508004F60670169016B016D016F01710173017501BB
S31508004F7077017A017C017E019201B103B203B30382
S31508004F80B403B503B603B703B803B903BA03BB033F
S31508004F90BC03BD03BE03BF03C003C103C303C403ED
S31508004FA0C503C603C703C803C903CA0330043104CB
S31508004FB03204330434043504360437043804390417
S31508004FC03A043B043C043D043E043F0440044104C7
S31508004FD04204430444044504460447044804490477
S31508004FE04A044B044C044D044E044F045104520425
S31508004FF053045404550456045704580459045A04CF
S315080050005B045C045E045F047021712172217321C4
S315080050107421752176217721782179217A217B21BE
S315080050207C217D217E217F2141FF42FF43FF44FFF2
S3150800503045FF46FF47FF48FF49FF4AFF4BFF4CFF26
S315080050404DFF4EFF4FFF50FF51FF52FF53FF54FFD6
S3150800505055FF56FF57FF58FF59FF5AFF00004100FA
S315080050604200430044004500460047004800490006
S315080050704A004B004C004D004E004F0050005100B6
S315080050805200530054005500560057005800590066
S315080050905A002100E0FFE1FFE5FFE2FFE3FFC00061
S315080050A0C100C200C300C400C500C600C700C800CE
S315080050B0C900CA00CB00CC00CD00CE00CF00D0007E
S315080050C0D100D200D300D400D500D600D800D9002C
S315080050D0DA00DB00DC00DD00DE00780100010201F9
S315080050E00401060108010A010C010E011001120152
S315080050F01401160118011A011C011E0120012201C2
S315080051002401260128012A012C012E013001320131
S315080051103401360139013B013D013F01410143019B
S31508005120450147014A014C014E0150015201540103
S31508005130560158015A015C015E0160016201640171
S31508005140660168016A016C016E01700172017401E1
S31508005150760179017B017D01910191039203930305
S315080051609403950396039703980399039A039B035D
S315080051709C039D039E039F03A003A103A303A4030B
S31508005180A503A603A703A803A903AA0310041104E9
S315080051901204130414041504160417041804190435
S315080051A01A041B041C041D041E041F0420042104E5
S315080051B02204230424042504260427042804290495
S315080051C02A042B042C042D042E042F0401040204A3
S315080051D003040404050406040704080409040A046D
S315080051E00B040C040E040F04602161216221632163
S315080051F06421652166216721682169216A216B215D
S315080052006C216D216E216F2121FF22FF23FF24FFD0
S3150800521025FF26FF27FF28FF29FF2AFF2BFF2CFF44
S315080052202DFF2EFF2FFF30FF31FF32FF33FF34FFF4
S3150800523035FF36FF37FF38FF39FF3AFF0000050212
S315080052400602060307030803090309040A040B04F4
S315080052500C040C050D050E050F050F0610061007A4
S31508005260100800000060000800200000030000008D
S3150800527000800008002000000400000000A00008CC
S31508005280002000000500000000C000080020000003
S315080052900600000000E000080020000007000000EB
S315080052A00000010800200000080000000020010896
S315080052B0002000000900000000400108002000004E
S315080052C00A00000000600108002000000B00000032
S315080052D000800108002000000C00000000A0010862
S315080052E0002000000D00000000C00108002000009A
S315080052F00E00000000E00108002000000F0000007A
S31508005300305400080000002048000000280100086A
S315080053107854000848000020801500004401000861
S315080053201001000043000000F8FFFFFF0040404066
S31508005330404040404040414141414140404040405A
S315080053404040404040404040404040404005020206
S3150800535002020202020202020202020202202020C5
S315080053602020202020202002020202020202909021
S31508005370909090901010101010101010101010101F
S315080053801010101010101010020202020202888873
S31508005390888888880808080808080808080808087F
S315080053A00808080808080808020202024000000067
S315080053B000000000000000000000000000000000DF
S315080053C000000000000000000000000000000000CF
S315080053D000000000000000000000000000000000BF
S315080053E000000000000000000000000000000000AF
S315080053F0000000000000000000000000000000009F
S31508005400000000000000000000000000000000008E
S31508005410000000000000000000000000000000007E
S31508005420000000000000000000000000000000006E
S31508005430000000000102030401020304060708092C
S315080054400204060801000000000000000000000039
S31508005450000000000400000000000000000000003A
S31508005460000000000000000000000000000000002E
S30D08005470000000000000000026
S705080000ED05
